:030000000219FDE5
:03000B000200AA46
:03002B000201804F
:03005B000203326B
:0300730002031F66
:1000800002030406080C10182030406080040608A3
:100090000C10182030406080A0C00003070F1F0D17
:1000A0000D0403060D0503030202C2AF306308C24C
:1000B0006385798AD2AF32C0D0C0E0206221E525C5
:1000C0006016E473E525F4C3334009758A00D263F2
:1000D000F57901D6F58AD262D0E0D0D0D2AF32C362
:1000E000E526334009758A00D263F57901F0F58A77
:1000F000C262E526F4603130682720720CE57BF49B
:100100005290D0E0D0D0D2AF32E57BF45290206F45
:100110001020650DE57BF4D33333335290E57B42F9
:1001200090D0E0D0D0D2AF32758A00D2637579001A
:10013000C28DD262212101C4306807206504D295A6
:10014000D29201C4306807206504D294D29101C4D0
:10015000306807206504D293D29001C4306807202C
:100160006504D295D29201C4306807206504D29408
:10017000D29101C4306807206504D293D29001C4A3
:10018000C2AFC2AD53E6EFC0D0C0E0D2D3D2AFE52C
:100190007A6009E57760057577004122757701C2BD
:1001A000CEE52A600720744F152A21F778007900E0
:1001B00020742EE580307E01F430E70278FF53DAB8
:1001C000CF207E0343DA20307E0343DA10C2D8C248
:1001D00071E580307E01F430E70279FFC3E8997061
:1001E000CB306103752A40207403752A40885CD2A5
:1001F00070E86003755F0020740DE52B6004152B1B
:10020000410743DA01C2D8207002411AA85C20617C
:1002100002C270207402411888227882B6040385D5
:10022000222420CF0AD0E0D0D043E610D2AD32C293
:10023000CF053AE57A6009E57860057578006115C3
:100240007578017802E52A6005307402152AC3E545
:100250005C94014005755F00416B75600075690035
:10026000E55F2401F55F5003755FFF7982B7020DEA
:10027000306E1DC3E52294324016854C227982B738
:10028000030E306E0BC3E52294324004798E872230
:10029000C3E5239522600840041523419F0523D818
:1002A000CA0569E56970021569D56A69756A0178D8
:1002B00008E56B60497805C3E569956B4057C3E570
:1002C00069956C50087801756A030202D9C3E56923
:1002D000956D50057801756A01C3E5629524401E4D
:1002E0007982B70402610A206E14852462E56904EC
:1002F0006003856B69756A0175233C020315E5622D
:100300002850057562FF610AF562E56204700675A2
:1003100060FF7569FFD0E0D0D043E610D2AD32C2A5
:10032000AF53E67F7592FA7593FFC260759104D260
:10033000AF32C2AF53E6EFC2ADC0D0C0E0C0F0D222
:10034000D3D2AFA8FBA9FCE57A6007C3E913F9E8AB
:1003500013F8C2D830710261A453DACF207E034370
:10036000DA10307E0343DA20D271E580307E01F46A
:1003700020E702617B88278928A18953DACF207E74
:100380000343DA20307E0343DA10C2D8C2713074DE
:1003900002A1757800E580307E01F430E702A17596
:1003A000885CA15D53DACF207E0343DA20307E03E0
:1003B00043DA10C271206102817D53DACF207E03BF
:1003C00043DA10307E0343DA20C2D8D271885789CD
:1003D00058C3E89555F8E99556F97B007E087A00F0
:1003E000C3E8948CE994005005755B00816F882107
:1003F00078A2E6A8216055C3E894C8E994005008A3
:10040000E4D2E4FB7A0A814AC3E89468E994015093
:1004100008E4D2E3FB7A0F814AC3E894D0E994025E
:100420005008E4D2E2FB7A1E814AC3E894A0E99422
:10043000055008E4D2E1FB7A3C814AC3E89498E98C
:1004400094085008E4D2E0FB7A787E00C3E895591E
:10045000FCE9955AFD30E70AECF42401FCEDF43494
:1004600000FD755B00C3EC9AED9E5003755B01883F
:0F04700059895A8557558558567802A15DC3E8BA
:10047F009527F8E99528F9307C02A141307B02A13C
:10048F0041307A02A13A20750281A0E9FDE8FC8192
:10049F00BFE9C313F9E813F8307902A13AE9C3139E
:1004AF00F9E813F8307802A13AE9C313FDE813FC19
:1004BF0020612CC3EC941CED9402400281D6ED70A8
:1004CF001EC3EC94C850180529E52970021529C3DD
:1004DF00E529940A5002A175755C00D270A175E5EB
:1004EF0029600215297400207F037896E624FAFE0E
:1004FF00E43400FFC3EC9EFCED9FFD5006780079BD
:10050F0000A141C3EC94FFED9400400678FF790001
:10051F00A141EC8572F0A4C5F0A2F733F879004041
:10052F000302055D78FF790002055DE9C313F9E861
:10053F0013F8307C0EE9600278FFC3E81338F8E453
:10054F003400F9C3E894FFE99400400278FF885C17
:10055F00D270206102A175741FF4552F4BF52FC275
:10056F0074EB7002D274752A40307403752A0A3006
:10057F006102A18920740353DAFE207403752B20C6
:10058F00D0F0D0E0D0D0D2AD43E6103279010205E1
:10059F00B979030205B9790A0205B9791E0205B9BD
:1005AF0079640205B979C80205B97817E4D5E0FD79
:1005BF00D8FAD9F6227A147B780205E07A107B8C70
:1005CF000205E07A0D7BB40205E07A0B7BC80205C9
:1005DF00E0E573D5E001227902E4C291D5E0FDD2C6
:1005EF0094D291D5E0FDC291D5E0FDC294D291D5C0
:1005FF00E0FDE920E004D295D29230E004D293D20C
:10060F0090E573D5E0FDE920E002C29230E002C22E
:10061F00907496D5E0FDD9C1EAF8D5E0FDD8FBDBA3
:10062F00B0C29122C37C007D0075F00005F0EA3363
:10063F00FAEB33FB50F6EB13FBEA13FAC3E9FFE8CF
:10064F00FEE89AF8E99BF95004EFF9EEF8B3EC33B2
:10065F00FCED33FDD5F0DFEDF9ECF822E889F08AF7
:10066F0020D2D4F8A9F07B0030F70B7BFFF42401E4
:10067F00F8E9F43400F9E88520F0A4ADF0F8E98545
:10068F0020F0A4AFF0FEED2EF974003FFA7C04C306
:10069F00EA13FAE913F9E813F8DCF48BF030F70AF0
:1006AF00E8F42401F8E9F43400F9E889F0C2D4F849
:1006BF00A9F0227882B60403020761C3E55C94199E
:1006CF00401EE52D54067018206E3678057994E794
:1006DF00146007780A1460027812C3E54198401F2E
:1006EF00306E098564627569FF756A01852224E49D
:1006FF00F544F545F546F547F548C26E020761D258
:10070F006E7994E7147013E523F43333F913F8E992
:10071F00540104F9E854FE020755E714147014E568
:10072F0023F4333333F913F8E9540304F9E854FC91
:10073F0002075DE523F433333333F913F8E9540734
:10074F000404F9E854F8C39440F8E99400F9884494
:10075F00894522C3E54113F9E54013F8C3E54498F1
:10076F00F8E54599F9500CC3E89480E994FF4016D9
:10077F00020799C3E8947FE9940050030207997820
:10078F007F7900020799788079FF8849894A22E5A5
:10079F00492546F8E54A3547F9854A20E4300701EF
:1007AF00F43548FA30E709C3EA94F040150207D749
:1007BF00C3EA940F50030207D778FF79FF7A0F022D
:1007CF0007D7780079007AF0C3E5249561500AC302
:1007DF0074019524500B0207F5E54A20E70E020736
:1007EF00F5E54A30E706884689478A482278A5E624
:1007FF00FAC3E54933F8E54A33F912066BE930E7F6
:10080F000BC3E89480E994FF40130130C3E8947F51
:10081F00E9940050020130787F79000130788079B7
:10082F00FFE820E715C3E52398F84009C3E89401D2
:10083F0040030208577801020857E8F424012523E2
:10084F00F8400302085778FF884B2278A6E6FAA8EB
:10085F0047A94812066BE930E70CC3E89401E99405
:0F086F00FF401602088CC3E894FFE99400500381
:10087E0002088C78FF790002088C780179FFE92054
:10088E00E715C3E54B98F84009C3E894014003020D
:10089E0008B378010208B3E8F42401254BF84003AD
:1008AE000208B378FF88242278FF20692879A1E70F
:1008BE006023E541601F74FF8541F0848539F03077
:1008CE006A0375F005A4F8C5F0600278FFC3E895D9
:1008DE00645002A864886322C3E54094C8E541943D
:1008EE0000E56350031401F7046002F56322788378
:1008FE00E6F520120FC675E89012059B75E890304C
:10090E00EDFDA8BDA9BE121087756E55756F00C39B
:10091E00740013FD7455606613FC74552CFC740042
:10092E003DFDECFAEDFBC3E89AE99B4014E56E241D
:10093E0055F56EE56F3400F56FEA2CFAEB3DFB8052
:10094E00E5AE6EAF6FC3E56F13F9E56E13F8C3E94D
:10095E0013F9E813F87A03C3E913F9E813F8DAF791
:10096E00AA201A7009756E00756F0002098C1AEABA
:10097E006008EE28FEEF39FFDAF88E6E8F6F227563
:10098E00E890227883E6FF30EDF9A8BDA9BE057088
:10099E00C3E57094084052757000E9FA79A0E760DB
:1009AE0044EA7007E571601B0209C5C3E8957160E2
:1009BE0010E5715006600C140209D10460F90209A9
:1009CE00D1E571F571C39472401B7561C0C3940477
:1009DE004013756180C39404400B756140C3940449
:1009EE00400375610075BB0E22EFC39401601F7446
:1009FE0055601BC3E894FFE994035012C3E8956E4B
:100A0E00E9956F5009E561600C1561020A23E561F5
:100A1E00F460020561A861C3E524985002A824C3BE
:100A2E00E89562400AA862E562F460038562618817
:100A3E00258826E570B4070375BB1022743279A79A
:100A4E0087F0A4C5F0A2F733F8C3E895614002A879
:100A5E00618822882488258826886422754000753E
:100A6E0041F022C2AF75C820A8CCA9CDAA3A30CF8A
:100A7E00010A75C824D2AFC3EA13FAE913F9E813D1
:100A8E00F8AB3BAC3C883B893CC3E89BF8E99C2027
:100A9E00690A547FF9306602619041EAAD3D8A3DA4
:100AAE00F9EA9D547FFA600678FF79FF41CFAE3E9A
:100ABE00AF3F8B3E8C3FA83BA93CC3E89EF8E99F15
:100ACE00F9C3E54113FBE54013FAE82AF540E93B8B
:100ADE00F54150067540FF7541FF6137AA40AB41A5
:100AEE00AC40AD417E047F02C3EB9404400D1E1F4B
:100AFE00C3EB94084005206A021E1FC3ED13FDECE4
:100B0E0013FCDEF7C3EA9CFAEB9DFBEF6009C3E929
:100B1E0013F9E813F8DFF7EA28FAEB39FB8A408B72
:100B2E004150067BFF8B408B41C3EB94025002D2A7
:100B3E00663069047F0361627892E6FFC3E53794FD
:100B4E008240110FC3E53794A040010FC3EF940606
:100B5E0040027F057E02E541C4540FF9E541C454BD
:100B6E00F0F8E540C4540F28F8C3E89EFAE9940063
:100B7E00FB4009C3EA9402EB940050047A02E4FBB2
:100B8E0061DCAA40AB41EBC4FEEAC4540F4EFCC379
:100B9E00EA9CFAEB9400FBC3E813C313F8EA28FAB5
:100BAE00EB3400FB8A408B41C3EB94024002C266D9
:100BBE007802EBC4FE7B00EAC4540F4EFAC3EA98E7
:100BCE00FA4005C3940250027A027892E6FF306032
:100BDE000261DC855192855293D26043E680C3E474
:100BEE009AF8E49BF9C3E833F8E933F930660281E9
:100BFE006FE8FAE9FBD3E913FDE813FC885189523B
:100C0E00C3EF94036038EF20E00DE82CF8E93DF9CE
:100C1E00ECFAEDFB020C38E828F8E939F9C3E824C0
:100C2E0002F8E93400F97AFE7BFFC3EF9403400E1D
:100C3E008A538B54884D894E8C4F8D5081A3885387
:100C4E0089548A4D8B4E8C4F8D503069127553F0EE
:100C5E007554FF754FF07550FF7551F07552FF8149
:0F0C6E00A3E8FAD3E813FC8851C3EF9403602086
:100C7D00EF20E007E82CF8ECFA818FE8282402F841
:100C8D007AFEC3EF940340088A53884D8C4F81A39D
:100C9D0088538A4D8C4FE568C3335002646BF568F9
:100CAD0030600281AD753402D26043E680E52D548B
:100CBD0006602DA840A941C3E913F9E813F830697E
:100CCD0004E92440F9C2AF53E67F759100C3E4985F
:100CDD00F594E499F595759104D26043E680D2AF11
:100CED0022D264754300752000306C0375204002DC
:100CFD000D0DD264754300752040306C03752000D6
:100D0D0078017901206620E52D54066002C26479D0
:100D1D0014E541C313700104F8C394144002781410
:100D2D00306904781B791BC3E833F8C3E933F92024
:100D3D006010E543600C306903D53404D26DA1C356
:100D4D0091B50543E59B5440B52002A1AD3069092D
:100D5D0008C3E899400118A13C20640A08C3E8992A
:100D6D004002A10DA13CC264C2AF53E67F75910054
:100D7D003066127594007595F0759104D26043E656
:100D8D0080D2AFA10DE5417EFFC3334009C333408F
:100D9D0005C3334001FEC3E49E759400F595A1860D
:100DAD00C3E53394015002A10D306402A10DD802A8
:100DBD00A1C1A13CC26DC2AF53E67F7591008553B1
:100DCD0094855495759104854D92854E93D26043CB
:100DDD00E680D2AFE52D54066008206A0205330285
:100DED000DFF306D0D206C0A2064071581158102F1
:100DFD0017002278003064027801E53775F007A4FA
:100E0D00F9E5F028F5F0E9A2F013A2F113A2F2131F
:100E1D00F537C394785003753778C3E53795384067
:100E2D0007D265E57BF45290306002C135854F9253
:100E3D00855093D26043E68022207D1AC2AF754261
:100E4D0002C291C295D292306204D293D290D2AFA7
:100E5D00759F11021084C2AF754202C291C293D226
:100E6D0090306204D295D292D2AF759F1102108448
:100E7D0030724B207D24C2AF754203900168757BA3
:100E8D0002C290C290306206D294D291C19FC29498
:100E9D00D291D2AF759F01021084C2AF75420390FB
:100EAD000168757B02C292C292306206D294D291D1
:100EBD00C1C3C294D291D2AF759F21021084207DFF
:100ECD001CC2AF754203900144757B02C290306223
:100EDD0004D294D291D2AF759F01021084C2AF7526
:100EED004203900144757B02C292306204D294D2C7
:100EFD0091D2AF759F21021084207D1AC2AF754229
:100F0D0004C292C293D290306204D294D291D2AFE5
:100F1D00759F21021084C2AF754204C290C295D252
:100F2D0092306204D294D291D2AF759F0102108497
:100F3D0030724B207D24C2AF75420590015C757BEC
:100F4D0004C291C291306206D295D292E15FC295F0
:100F5D00D292D2AF759F11021084C2AF7542059027
:100F6D000174757B01C291C291306206D293D29009
:100F7D00E183C293D290D2AF759F11021084207D70
:100F8D001CC2AF754205900138757B04C291306269
:100F9D0004D295D292D2AF759F11021084C2AF7553
:100FAD004205900150757B01C2913062E8D293D217
:100FBD0090D2AF759F11021084207D1AC2AF754279
:100FCD0006C290C294D291306204D295D292D2AF21
:100FDD00759F01021084C2AF754206C292C294D2AF
:100FED0091306204D293D290D2AF759F21021084BA
:100FFD0030724C207D24C2AF754201900174757B17
:10100D0001C292C292306206D293D290011FC29356
:10101D00D290D2AF759F21021084C2AF754201905C
:10102D00015C757B04C290C290306207D295D2925A
:10103D00021044C295D292D2AF759F010210842046
:10104D007D1CC2AF754201900150757B01C292307B
:10105D006204D293D290D2AF759F21021084C2AF99
:0E106D00754201900138757B04C29030620418
:10107B00D295D292D2AF759F01C26522900136757F
:10108B007B00C292C291C290C292C291C290C262C4
:10109B0022788076070876070876010876040876AA
:1010AB00FF0876FF08760A087602087601087601B3
:1010BB00788C76010876000876B40876FF0876FF00
:1010CB000876FF0876030876FF0876010876FF0896
:1010DB0076250876D00876780876C80876040876E0
:1010EB00FF08760108760008767A08760A087601FA
:1010FB000876010876000876FF087600227887E6E6
:10110B00FFC272BF0302D2727888C27DE630E10261
:10111B00D27DC27E7889E630E102D27EC3EF9402A3
:10112B006008758E01D27302113A758E00C273225C
:10113B007880E6149000809378A5F67881E6149079
:10114B0000809378A6F67886E61490008D9378A7A6
:10115B00F6789FE6F87005756B002181C3E8941152
:10116B0040027811E82828F56B256B256B28F56C68
:10117B00256B2828F56D7886E6F539C39402500364
:10118B00753902789CE67538FFB402037538A0B444
:10119B00030375388278A3E61490009A93F56611D1
:1011AB008722227896E6FA7897E6FB7888E6B403EE
:1011BB0005C3EB940EFB307F047A007BFFC3EB9AE5
:1011CB00FCC3948250027C827572000572EC8572AE
:1011DB00F0A4C3E5F0947D40F222D27F31AE12052C
:1011EB00AA1205AA7A007B007C101205A0E55C2AE6
:1011FB00FA74003BFBDCF37C04C3EB13FBEA13FA3E
:10120B00DCF7FEC27F31AE22757C00757D00E5EF09
:10121B0020E6037520000520903FFFE520146006B3
:10122B00901FFF1460009304600375EF1653D9BF32
:10123B007581C043FF8012059B75EF0643B203E532
:10124B00B3240220E70DF521E5E320E0068521B369
:10125B0043E30111877580FF75A40075F19175D477
:10126B007F75900075A53F75F23F75D50075A6018A
:10127B0075E2411187E4F8F6D8FD756801119C12EF
:10128B00176478988673753001C2AF1205B41205D6
:10129B00C41205AA1205CB1205AA1205D21205AA71
:1012AB0012189A1205B41205B41205AFC2AF757CB1
:1012BB0000757D0078FA79FA308707D9FBD8F702E9
:1012CB001C003108313B31AD31AE789886731187F4
:1012DB0075A90075B680757A0075881075890275C9
:1012EB00C82475910475D84075A82275B80275E6A7
:1012FB0090759B80759D0075D10E75BCC075BB0E2E
:10130B0075BA1175E88012059BD2AF1208FC7536C1
:10131B000053DACF207E0343DA20307E0343DA100A
:10132B0043DA01C2D8C2711205B4D2617B037A0CC5
:10133B00E55B70077A0CDB030212B71205AA20706B
:10134B00030212B7C270E55CC3940240E1E52F546F
:10135B001F855E5DF55EB55DD5DAD5C26153DACF1B
:10136B00207E0343DA20307E0343DA10C2D8C271E9
:10137B0078A2E67008D274E52F54E0F52FC275758C
:10138B0029001205AF307409C3E529940A4002D233
:10139B00751205A078023074027800C3E55C9840A2
:1013AB00F0C2AF1205C41205C41205C4D2AF1205A8
:1013BB00B4754C001205A0788CE6C394015003025F
:1013CB0014ACE530C3940150030214AC757CA575C5
:1013DB007DF1207435C3E55C94FF50030214ACC25D
:1013EB00AF1205D9D2AF1205AFC3E55C940150EF34
:1013FB00C2AF1205C41205A51205C4D2AF1205AFB8
:10140B00C3E55C94FF40E902191F7F05D27F31AE23
:10141B001205AFC2AFC27F31AEAE5CC3E55C947F49
:10142B00D2AF500281BC12059BC2AF1205D9D2AF0D
:10143B00DFDA31E5C3EE94057897F61205B412188E
:10144B00A27F0AD27F31AE1205AFC2AFC27F31AEDF
:10145B00AE5CC3E55C947FD2AF50E612059BC2AF86
:0F146B001205C41205A51205C4D2AFDFD631E5B4
:10147A00EE24037896F6F87997E7C39482400398A6
:10148A005006E824827897F61205B41217B112189A
:10149A00D11205AF31AEC3E55C94FF500261D702A9
:1014AA00191F757C00757D00C3E55C954C4003856A
:1014BA005C4C1205AF78017988E7B403027805C35A
:1014CA00E55C98400261BFC2AF1205D91205D91274
:1014DA0005D9D2AF1205B4753000E4F531F53205FD
:1014EA0031E531F4703E0532789AE67819146012C3
:1014FA00783214600D787D14600878FA14600375E8
:10150A003200C3E53298401C118712059B153275CB
:10151A00310078998673C2AF1205D9D2AF7898860E
:10152A00731205AF1205A5E52A700530740241B79A
:10153A0078012074027806C3E55C9840A21205AFD0
:10154A00E52A70030212B7C2AF1187E4F522F52328
:10155A00F524F525F526F567D2AF7885E6C333F588
:10156A0065E4F544F545F546F547F548F570F52C7B
:10157A00F52DF53775700875BB1012059B12098D8C
:10158A0030EDFDA8BDA9BEE97001F8887112099174
:10159A0075700875BB103108C2AF7561FF120A4A2F
:1015AA00852261852262852263D2AF752201752464
:1015BA0001752501752601856069756A0175B69000
:1015CA0075A903757A017888E6B40307C27D307677
:1015DA0002D27DD268D269753300120FC6120FFD8E
:1015EA00120A6A120A71120A6A120A71120A6A1233
:1015FA000CFF1206C2120E00120E46120A71120CCB
:10160A00EE306E031207622066031208B6306603D4
:10161A001208E6120E00120E7D120A71120CFF3029
:10162A006E0312079E120E00120F06120A71120C96
:10163A00EE306E031207FC120E00120F3D120A71F1
:10164A00120CFF306E0312085A120E00120FC61245
:10165A000A7112098D120CEE120E00120FFD1209F8
:10166A0091120A7130692C856461856462856069AA
:10167A00756A0179187A0CC3E533994009C269D2AF
:10168A006A8A3502169DC3E55C940140030215F986
:10169A00021708306A25206C22E535147006C26AE2
:1016AA00D26BA1F9F535C3E55C940140030215F943
:1016BA007888E6C394036003021708753600C3E509
:1016CA005F94014009856462856069756A0178FAE8
:1016DA0079A4E760027803C3E55F98502130740467
:1016EA00E52A601A78F0306C058564617820C3E5D4
:1016FA0041985002A1F90536E55C6002E10B7536A6
:10170A0000C2AF11877887E6FE760231087887EE45
:10171A00F6E4F522F523F524F525F526F565752C6D
:10172A0000752D0075A90075B680757A00D2AF12C2
:10173A0005AF118778A4E6600CC295D292C294D202
:10174A0091C293D290307406E52A700241B7788D1F
:10175A00E6C394014002619C81E4901A0D7820123C
:10176A0017F3E520B4A50CA31217F3E520B45A0326
:10177A00021791757CA5757DF1119C1217B1757CC4
:10178A0000757D000217B0901A0378807B0A121741
:10179A00F3A308DBF9901A0F788C7B191217F3A3BD
:1017AA0008DBF9901A2822C2AF12183812181390BF
:1017BA001A00740E1217F8A374091217F8A37415F5
:1017CA001217F8901A0378807B0A1217F7A308DB1E
:1017DA00F9901A0F788C7B191217F7A308DBF91204
:1017EA00184C121827901A2822E493F622E6438FFF
:1017FA0001538FFDFFC3E583941C400122EF857CD2
:10180A00B7857DB7F0538FFE22438F02438F018540
:10181A007CB7857DB7901A0DF0538FFC22901A0D74
:10182A0074A51217F8901A0E745A1217F8227A3001
:10183A0079D07820901A401217F3E520F709A3DA35
:10184A00F6227A3079D0901A40E71217F809A3DA0B
:10185A00F822AB74A875BB01027980BB02027981B8
:0F186A00BB03027982BB04027994BB0502798328
:10187900BB06027986BB07027992BB08027987BB4E
:101889000902799CBB0A027988BB0B027989E8F7BE
:10189900227C051205B4DCFB22C2AF1205C4120575
:1018A900CB1205D21205D91205A51205C41205CB12
:1018B9001205D21205D91205A51205C41205CB12BB
:1018C90005D21205D9D2AF22C2AF1205D91205D25B
:1018D9001205CB1205C41205A51205D91205D2129B
:1018E90005CB1205C41205A51205D91205D2120598
:1018F900CB1205C4D2AF22AE74AF75C2AF1205C404
:101909001205C41205C41205A5DEF21205D9120585
:10191900A5DFF8D2AF2211A2119A119A7574017537
:10192900750175760031007C05AD5C1205B4C3ED17
:10193900955C70F5C3E55C9401400AC3E55C94FFCE
:10194900403302195C115C1217B111A2C2AF75EFD5
:1019590016119ADCD40576C3E5769403500280C546
:10196900119A0575E5741490009F93F808C3E575FD
:1019790098500280AD119A119A0574C3E574940CBC
:101989005002809B12109C1217B1C2AF75EF16114D
:011999009AB3
:0319FD00021213C0
:101A00000E091507070104FFFF0A020101A55A018B
:101A100000B4FFFFFF03FF01FF25D078C804FF01DA
:091A200000FF0A010100FF00FFB4
:101A400023454D41585F4C746E675F32304123200F
:101A500023424C48454C492346333930232020202B
:101A60002020202020202020202020202020202076
:101C0000C2AFC2D353D9BF7581C043B20343FF8073
:101C1000752438752503B1DC7529A5752AF175E29F
:101C20004043F18053A47F75D4FFD2877DFA7803B7
:101C300079E67C10752200752300901DE97B0675FE
:101C400024987525013087028145208708D8FBD963
:101C5000F9DCF781B7308708D8FBD9F9DCF781B711
:101C6000B19CE493A3C39A6004DDC381B7DBDBB10D
:101C70008E6002812E7B08E493FAA3B16FDBF87AC1
:101C800030B16F752200752300B18EEAFCEBFDC305
:101C9000ED94FE400EB18E8A278B28ED30E0048A49
:101CA000828B83B18E7AC270D8C3ED94FE601950D6
:101CB000CEBD002BEC600F7520007521FF7529004B
:101CC000752A000200008100A827A9280809D80465
:101CD000D90281DCB192EA89AAF281CE0D81A3C337
:101CE000ED94035053EDA2E092007AC5C3E58294CF
:101CF00000E583941C508A200010438F02438F011B
:101D00008529B7852AB7F0300029A827A92808090E
:101D1000438F01538FFDD804D902A133C3E58394C7
:101D20001C4003A3A11689AAE28529B7852AB7F02A
:101D3000A3A116538FFC817F7AC1BD030CE493A34A
:101D4000FAB153DCF8B14B817F8181AA22AB23B178
:101D50006FEBFAEA6222752608C3E52313F523E543
:101D60002213F52250066323A0632201D526EAB18F
:101D7000DCB1DC75260AEAF4200102D287300102C8
:101D8000C287B1DCC3134002C201D526EB22B19257
:101D9000EAFB208702A192308702A197752608AE40
:101DA00024AF25C3EF13FFEE13FEB1E0B1DCC3EAAD
:101DB000133087024480FA30E703632201C3E5232E
:101DC00013F523E52213F52250066323A0632201B5
:101DD000D526D9E52265236523F52222AE24AF2539
:101DE0000E0FDEFEDFFCD20122424C48656C6934E6
:071DF000373164F390060196
:00000001FF
